:020000040800F2
:100000000010002095180008B1040008BD04000885
:1000100000000000000000000000000000000000E0
:10002000000000000000000000000000C104000803
:100030000000000000000000CD040008D904000802
:10004000E118000800000000E1180008E1180008AD
:10005000E1180008E1180008E1180008E11800089C
:1000600000000000930700085D0A0008E11800087E
:10007000E1180008E1180008E1180008000000007D
:10008000E11800080000000000000000E11800086E
:1000900000000000F5030008E1180008E11800085E
:1000A00000000000C903000800000000E11800087B
:1000B0000000000000000000000000000000000040
:1000C00080B582B000AF0200FB1D1A70FB1D1B78CB
:1000D0001A001F231A40044B012191400A001A60A4
:1000E000C046BD4602B080BD00E100E090B583B0DF
:1000F00000AF02003960FB1D1A70FB1D1B787F2BBF
:1001000032D92F4AFB1D1B7819000F230B40083BE7
:100110009B0806339B00D31804331B68FA1D127822
:10012000110003220A40D200FF2191400A00D2436D
:100130001A4011003B689B01FF221A40FB1D1B78EF
:10014000180003230340DB009A401D48FB1D1B7869
:100150001C000F232340083B9B080A4306339B00E7
:10016000C31804331A6027E0164AFB1D1B785BB2E4
:100170009B08C0339B009B58FA1D12781100032284
:100180000A40D200FF2191400A00D2431A401100D8
:100190003B689B01FF221A40FB1D1B7818000323BC
:1001A0000340DB009A400748FB1D1B785BB29B08AD
:1001B0000A43C0339B001A50C046BD4603B090BDF1
:1001C00000ED00E000E100E080B582B000AF7860B3
:1001D0007B685A1E80235B049A4201D3012310E0FE
:1001E0000A4B7A68013A5A6001235B4203211800E6
:1001F000FFF77CFF054B00229A60044B07221A6030
:1002000000231800BD4602B080BDC04610E000E0EB
:1002100080B500AFC046BD4680BD80B582B000AF9E
:100220005B4B1A685A4B802149020A431A60C04648
:10023000574B1A6880239B021340F9D0544B5A68DD
:10024000534B54490A405A60514B5A68504B8821CD
:1002500049030A435A604E4B1A684D4B80214904AA
:100260000A431A60C0464A4B1A6880239B04134015
:10027000F9D0474B5A68464B02210A435A6000F0B6
:1002800011FE454B1B680A21180001F08DF903008F
:100290001800FFF799FF01235B421800FFF710FFDA
:1002A00001235B4260211800FFF720FF384B5A6999
:1002B000374B3A490A435A61354B9A69344B3849AE
:1002C0000A439A61324BDA69314B02210A43DA61FF
:1002D0009023DB051A689023DB0532490A431A6034
:1002E0009023DB059A689023DB052F490A439A6027
:1002F0009023DB0500221A629023DB05882252003E
:100300005A622A4A294B12681A60294BC922920064
:100310001A60274BE022D2005A60254B1A68244B02
:1003200040210A431A601920FFF7CAFE4021192014
:10033000FFF7DCFE1F4B00225A601E4B0122DA60E1
:100340001C4B2F229A621B4B1B4ADA62194B01226B
:100350001A601520FFF7B4FE40211520FFF7C6FEF6
:10036000164B180000F05AF900F0BEFA144B3B602F
:100370003B680821180000F091FB00237B6002E03D
:100380007B6801337B607B680E4A9342F8DDEDE7C2
:10039000001002400CF8C3FF00000020110006000E
:1003A000015A420070A92800808A08000004004811
:1003B0000030014000440140E703000040420F00CC
:1003C000E41800089F86010080B500AF084B9B68C9
:1003D0000222134009D09023DB0508229A61044BC6
:1003E0005A68034B80218A435A60C046BD4680BD8F
:1003F0000030014080B582B000AF284B1B6901225C
:10040000134047D0254B1A69244B01218A431A61B6
:10041000FB1D00221A70BB1D01221A7000233B60D5
:100420001DE01F4B3A689200D358002B0FD01C4B95
:100430003A689200D358591E194B3A689200D1502D
:10044000FB1DF91DBA1D097812780A431A70BA1DEE
:10045000BB1D1B78DB1813703B6801333B603B68A6
:10046000072BDED90F4B1B68591C0E4A11600A2B53
:1004700010D10C4B00221A600B4AFB1D1B78137025
:100480000A4B5A68094B80210A435A609023DB05C6
:1004900008229A62C046BD4602B080BD00440140B9
:1004A000A8000020980000200C30014000300140DE
:1004B00080B500AF00BEC046BD4680BD00BEC04690
:1004C00080B500AF00BEC046BD4680BD80B500AF60
:1004D00000BEC046BD4680BD80B500AF0A4B1B685C
:1004E000591C094A11600A2B0AD1074B00221A60D5
:1004F000064B1B685A1C054B1A60054B64229A6117
:10050000C046BD4680BDC0469C000020940000202F
:10051000A800002080B582B000AF0200FB1D1A7059
:10052000FB1D1B781A001F231A40044B0121914028
:100530000A001A60C046BD4602B080BD00E100E07E
:1005400090B583B000AF02003960FB1D1A70FB1D2F
:100550001B787F2B32D92F4AFB1D1B7819000F23E4
:100560000B40083B9B0806339B00D31804331B68E1
:10057000FA1D1278110003220A40D200FF21914097
:100580000A00D2431A4011003B689B01FF221A4027
:10059000FB1D1B78180003230340DB009A401D4815
:1005A000FB1D1B781C000F232340083B9B080A43BC
:1005B00006339B00C31804331A6027E0164AFB1D5C
:1005C0001B785BB29B08C0339B009B58FA1D1278C6
:1005D000110003220A40D200FF2191400A00D243B9
:1005E0001A4011003B689B01FF221A40FB1D1B783B
:1005F000180003230340DB009A400748FB1D1B78CB
:100600005BB29B080A43C0339B001A50C046BD46EC
:1006100003B090BD00ED00E000E100E080B584B0E3
:1006200000AF78608023DB00180000F04BF8214B0E
:10063000802212061A611F4B07225A611D4B1E4A67
:10064000DA601C4B04229A621A4B9A68194B80217B
:1006500009060A439A60C046164B9B68002BFBDBD9
:10066000144B9A68134B01210A439A60114B9A6804
:10067000104B04210A439A607B68104A934206DDBE
:100680007B68FA21180001F019F8030000E0062346
:10069000FB60FA6880235B029A4201DB084BFB6037
:1006A000FB6819000C2000F03DF8C046BD4604B0C0
:1006B00080BDC0460024014043080000DC05000066
:1006C000FFFF000080B582B000AF7860114B124A86
:1006D0009A60104B114ADA600E4B7A685A600D4BE3
:1006E00000221A600B4B1A680A4B0D490A431A6024
:1006F0000920FFF70FFF40210920FFF721FF054BDD
:100700001A68044B01210A431A60C046BD4602B074
:1007100080BDC0460800024040240140C8000020BF
:10072000A205000080B582B000AF78603960154B3B
:10073000802212025A64134BC022D201DA61114B9B
:10074000802252011A620F4B01221A647B685A1EE2
:100750000C4B9A623B685A1E0A4BDA62094B5A6983
:10076000084B01210A435A61064B80221A60054B4F
:100770001A68044B01210A431A60C046BD4602B004
:1007800080BDC046002C014080B500AFC046BD46CC
:1007900080BD80B500AF054B5A68044B01210A4368
:1007A0005A60FFF7F1FFC046BD4680BD0000024021
:1007B00080B582B000AF0200FB1D1A70FB1D1B78D4
:1007C0001A001F231A40044B012191400A001A60AD
:1007D000C046BD4602B080BD00E100E080B582B0F9
:1007E00000AF0200FB1D1A70FB1D1B781A001F23AF
:1007F0001340054901229A40130080228B50C046C5
:10080000BD4602B080BDC04600E100E090B583B0B7
:1008100000AF02003960FB1D1A70FB1D1B787F2B97
:1008200032D92F4AFB1D1B7819000F230B40083BC0
:100830009B0806339B00D31804331B68FA1D1278FB
:10084000110003220A40D200FF2191400A00D24346
:100850001A4011003B689B01FF221A40FB1D1B78C8
:10086000180003230340DB009A401D48FB1D1B7842
:100870001C000F232340083B9B080A4306339B00C0
:10088000C31804331A6027E0164AFB1D1B785BB2BD
:100890009B08C0339B009B58FA1D1278110003225D
:1008A0000A40D200FF2191400A00D2431A401100B1
:1008B0003B689B01FF221A40FB1D1B781800032395
:1008C0000340DB009A400748FB1D1B785BB29B0886
:1008D0000A43C0339B001A50C046BD4603B090BDCA
:1008E00000ED00E000E100E080B500AF174B012211
:1008F00052421A60154B00225A60144B00229A6033
:10090000134B144A9A60124B92221A600A20FFF786
:100910004FFF20210A20FFF779FF0F4B0F4A1A6083
:100920000D4B3022DA600C4BC02292025A600A4B07
:100930009A68094B80210A439A60074B1A68064B54
:1009400001210A431A60C046BD4680BDC808002088
:100950001C00024028380140003801402C200000D3
:1009600080B584B000AF194BBB60BB685B687B602F
:10097000BB689B687A689A4205D2BB689A687B68B4
:10098000D31AFB6004E07B6880225200D31AFB601C
:10099000BB687A681A607A68FB68D318FF221A402D
:1009A000BB685A60BB680C331A007B68D218084BCE
:1009B000DA60074BFA685A60054B1A68044B01214C
:1009C0000A431A60C046BD4604B080BDC808002076
:1009D0001C00024080B582B000AF78600A00FB1CAA
:1009E0001A700A20FFF7FAFE7B689A687B681B681A
:1009F0009A4205D10A20FFF7DBFE10235B4211E08B
:100A00007B689B687A68D318FA1C12781A737B6823
:100A10009B680133FF221A407B689A600A20FFF727
:100A2000C7FE00231800BD4602B080BD80B582B06D
:100A300000AF0200FB1D1A70C046FB1D1A78064B62
:100A400011001800FFF7C6FF03001033F5D0C046B1
:100A5000C046BD4602B080BDC808002080B500AFCA
:100A60000B4B5A680A4B20210A435A60094B1A68FB
:100A7000084B01218A431A60074B9A68064B5B6852
:100A80009A4201D0FFF76CFFC046BD4680BDC0460C
:100A9000000002401C000240C808002080B582B05F
:100AA00000AF786039603A687B681100180000F088
:100AB00070F8054B1B680122134001D1FFF750FF6E
:100AC000C046BD4602B080BD1C00024080B588B063
:100AD00000AFF860B9607A603B60BA6880235B025F
:100AE0009A4202D23B68FE2B02D901235B424CE0C2
:100AF0003B680233BA689A4202D201235B4244E067
:100B00000023FB6136E0FB69002B0FD0FB69013B42
:100B10007A68D3181B78002B08D0FB69013B7A68F0
:100B2000D2181B23FB1812781A7019E0FB697B613D
:100B300002E07B6901337B617A693B689A4205D2A6
:100B40007A687B69D3181B78002BF2D17B69DAB203
:100B5000FB69DBB2D31ADAB21B23FB1801321A701D
:100B6000FA68FB69D3181B22BA1812781A70FB694D
:100B70000133FB61FA693B689A42C4D9FA68FB69A0
:100B8000D31800221A703B6802331800BD4608B023
:100B900080BD80B586B000AF786039603B68FE2BC1
:100BA00002D901235B4240E000237B6135E07B6991
:100BB000002B0FD07B69013B7A68D3181B78002B80
:100BC00008D07B69013B7A68D2181323FB1812788E
:100BD0001A7019E07B69FB6002E0FB680133FB607F
:100BE000FA683B689A4205D27A68FB68D3181B788A
:100BF000002BF2D1FB68DAB27B69DBB2D31ADAB22E
:100C00001323FB1801321A701323FB181B781800EA
:100C1000FFF70CFF7B6901337B617A693B689A427D
:100C2000C5D90020FFF702FF00231800BD4606B01B
:100C300080BD80B588B000AFF860B9607A603B6075
:100C4000BA6880235B029A4204D23A6880235B022E
:100C50009A4202D301235B4252E03B68002B02D14F
:100C600001235B424CE0BA683B689A4202D20123FE
:100C70005B4245E00123FB617B681B78BB61BB697C
:100C8000002B24D102235B423AE0BB69013BBB61EC
:100C9000BB69002B09D17A68FB69D3181B78BB614B
:100CA0001723FB1800221A7006E07A68FB69D21835
:100CB0001723FB1812781A70FB69013BFA68D318E6
:100CC0001722BA1812781A70FB690133FB61FA69AE
:100CD0003B689A4205D27A68FB69D3181B78002BCF
:100CE000D3D1FA693B689A4202D102235B4207E002
:100CF000BB69012B02D003235B4201E0FB69013B8E
:100D00001800BD4608B080BD80B582B000AF7860E5
:100D10007B6800221A607B6800225A60C046BD468C
:100D200002B080BD80B588B000AFF860B9607A606D
:100D30001A00FB1C1A70FB681B68002B0ED1FB1CF1
:100D40001B78002B54D0FB1C1A78FB685A60FB6898
:100D50001B685A1CFB681A60002350E0FB1C1B78C0
:100D6000002B0DD1FB685B68012B39D1FB681B6838
:100D7000013B7B61FB681800FFF7C6FF7B693EE023
:100D8000FB685B685A1EFB685A60FB685B68002B57
:100D900008D1FB1C1A78FB685A601F23FB1800223D
:100DA0001A7004E01F23FB18FA1C12781A70FB68F3
:100DB0001B68013BBB61BA697B689A4202D302237C
:100DC0005B421CE0BA68BB69D3181F22BA181278BC
:100DD0001A70FB681B685A1CFB681A6000230EE03F
:100DE000C046FB681800FFF78FFF01235B4206E057
:100DF000C046FB681800FFF787FF03235B4218001B
:100E0000BD4608B080BD0419000800000020940011
:100E1000002094000020D4090020000080B500AF1D
:100E20001A4B1A68194B01210A431A60174B5A686A
:100E3000164B17490A405A60144B1A68134B154950
:100E40000A401A60114B1A68104B13490A401A6085
:100E50000E4B5A680D4B11490A405A600B4BDA6A27
:100E60000A4B0F218A43DA62084B1A6B074B0C4975
:100E70000A401A63054B5A6B044B01218A435A639B
:100E8000024B00229A60C046BD4680BD0010024061
:100E90000CB8FF08FFFFF6FEFFFFFBFFFFFFC0FFE0
:100EA000ECFEFFFF80B584B000AF0023FB600023A1
:100EB000BB6000237B6000233B60314B5B680C22EE
:100EC0001340FB60FB68082B11D0FB68082B41D84E
:100ED000FB68002B03D0FB68042B04D03AE0294BBD
:100EE000294A1A603AE0274B274A1A6036E0244B19
:100EF0005A68F0239B031340BB60214B5A68802340
:100F00005B0213407B60BB689B0C0233BB601C4BD5
:100F1000DB6A0F22134001333B607A6880235B0257
:100F20009A420AD13968184800F03EFB03001A00C3
:100F3000BB685A43134B1A6010E0B9680A005201AB
:100F4000521A93019B1ADB005B181B021A000D4B0F
:100F50001A6003E00B4B0C4A1A60C046084B5B68F2
:100F60001B090F221340094AD35CFB60054B1A682A
:100F7000FB68DA40034B1A60C046BD4604B080BD32
:100F8000001002400000002000127A00EC18000857
:100F900080B500AF044B1A68034B8021C9020A4395
:100FA0001A60C046BD4680BD0010024080B500AF4B
:100FB000044B1A68034B04490A401A60C046BD46F8
:100FC00080BDC04600100240FFFFFBFF80B500AFB0
:100FD000044B1A68034B802149020A431A60C04639
:100FE000BD4680BD0010024080B500AF064B1A68B8
:100FF00080239B021340054A944663445A4253415E
:10100000DBB21800BD4680BD001002400000FEFFAC
:1010100080B500AF044B1A68034B01210A431A60E4
:10102000C046BD4680BDC0460010024080B500AF3E
:10103000054B1B6802221340023B5A425341DBB26C
:101040001800BD4680BDC0460010024080B582B089
:1010500000AF7860064B5B68032293431900044B92
:101060007A680A435A60C046BD4602B080BDC04699
:101070000010024080B500AF034B5B680C221340A8
:101080001800BD4680BDC0460010024080B582B049
:1010900000AF7860064B5B68F02293431900044B65
:1010A0007A680A435A60C046BD4602B080BDC04659
:1010B0000010024080B582B000AF7860064B5B68DC
:1010C000064A13401900044B7A680A435A60C04626
:1010D000BD4602B080BDC04600100240FFF8FFFFD1
:1010E00080B500AF044B1A68034B802149040A43C2
:1010F0001A60C046BD4680BD0010024080B500AFFA
:10110000074B1A6880239B041340FE221206944664
:1011100063445A425341DBB21800BD4680BDC0460D
:101120000010024080B582B000AF786039600E4B8D
:101130005B680E4A134019007A6880235B021A40EC
:101140003B681A43084B0A435A60074BDB6A0F227D
:10115000934319007B680F221A40034B0A43DA625B
:10116000C046BD4602B080BD00100240FFFFC2FF76
:1011700080B582B000AF786039603968786800F077
:1011800013FA03001A00064B013A5A60044B00227E
:101190009A60034B05221A60C046BD4602B080BD6E
:1011A00010E000E080B582B000AF7860064B1B68AD
:1011B000012293431900044B7A680A431A60C0461F
:1011C000BD4602B080BDC0460020024080B500AFE1
:1011D000034B1B68012213401800BD4680BDC0466A
:1011E0000020024080B582B000AF7860FA239A00F8
:1011F0007B6811001800FFF7BBFFC046BD4602B078
:1012000080BD80B584B000AF78600E4B1B68FB607A
:10121000FB687B6801330CD07B6801337B6008E09E
:10122000084B1A6880235B02134002D07B68013BA5
:101230007B607B68002BF3D1C046C046BD4604B03E
:1012400080BDC04610E000E080B582B000AF78609D
:10125000034B7A681A60C046BD4602B080BDC046E6
:101260000000002090B585B000AF786039600F2392
:10127000FB1801221A700023BB6000F0D4F80300B1
:10128000012B28D17B6801225A607B68174A19001C
:10129000100000F0ABF80300BB60FFF7C7FE0300CF
:1012A000012B07D0FFF7B4FEC046FFF7BFFE0300D7
:1012B000012BFAD17B681B6819000020FFF732FF71
:1012C0000F23FC183A68BB681100180000F0BEF844
:1012D0000300237003E00F23FB1800221A700F2372
:1012E000FB181B781800BD4605B090BD00127A00AF
:1012F00090B587B000AFF860B9607A603B601723A3
:10130000FB1801221A7000233B6100F08CF80300E7
:10131000012B32D17A68FB681100180000F066F8E2
:1013200003003B61FFF760FE0300012B0FD0BB6899
:10133000012B02D1FFF72CFE01E0FFF737FEFFF78C
:1013400045FEC046FFF750FE0300012BFAD17B6833
:101350005B68802252021A437B681B6819001000E8
:10136000FFF7E0FE1723FC183A683B6911001800EC
:1013700000F06CF80300237003E01723FB18002231
:101380001A701723FB181B781800BD4607B090BDD4
:1013900080B584B000AF78600F217B1801221A70ED
:1013A0000023BB607B68002B03D17B1800221A70DE
:1013B00013E07B680C4A934201D90123BB60BB68F0
:1013C0001800FFF7EFFEFFF701FF0200BB68934232
:1013D00003D00F23FB1800221A700F23FB181B7871
:1013E0001800BD4604B080BD00366E0180B584B0E3
:1013F00000AF786039600023FB603B685B680133B5
:101400001900786800F0D0F8030019003B681B68E9
:101410009B0C0F22134002334B43FB60FB68180008
:10142000BD4604B080BD80B582B000AFFB1D012277
:101430001A70FFF763FE031E02D0FB1D00221A7014
:10144000FB1D1B781800BD4602B080BD90B585B06D
:1014500000AF786039600F203B1801221A7000231A
:10146000BB602E4B1A683B681B681B090F210B40A1
:101470002B49CB5C9A401300BB60BA687B689A42E8
:1014800006D23C187B681800FFF782FF0300237028
:101490000F23FB181B78012B1AD1FFF721FEC04642
:1014A000FFF72CFE0300012BFAD13B681B681800E4
:1014B000FFF7ECFD0220FFF7C9FDC046FFF7DAFD9C
:1014C0000300082BFAD13B685B681800FFF7F2FDB8
:1014D000BA687B689A4207D90F23FC187B6818000A
:1014E000FFF756FF030023700F23FB181B78012B17
:1014F0000CD13B681B681B090F221340084AD35CC0
:101500001A007B68D3401800FFF79EFE0F23FB18DC
:101510001B781800BD4605B090BDC04600000020F5
:10152000EC18000880B500AFC046BD4680BD80B550
:1015300086B000AFF860B9607A60FA687B68D3184B
:101540003B61FB687B6106E0BB68DAB27B691A70BD
:101550007B6901337B617A693B699A42F4D3FB680A
:101560001800BD4606B080BD80B584B000AF78607D
:101570007B68FB60C0467B685A1C7A601B78002B36
:10158000F9D17A68FB68D31A013B1800BD4604B054
:1015900080BD80B582B000AF0200FB1D1A70C0464E
:1015A000BD4602B080BD0000002243088B4274D3C8
:1015B00003098B425FD3030A8B4244D3030B8B4254
:1015C00028D3030C8B420DD3FF22090212BA030C5D
:1015D0008B4202D31212090265D0030B8B4219D33E
:1015E00000E0090AC30B8B4201D3CB03C01A52415E
:1015F000830B8B4201D38B03C01A5241430B8B42A6
:1016000001D34B03C01A5241030B8B4201D30B038E
:10161000C01A5241C30A8B4201D3CB02C01A5241B5
:10162000830A8B4201D38B02C01A5241430A8B4278
:1016300001D34B02C01A5241030A8B4201D30B0261
:10164000C01A5241CDD2C3098B4201D3CB01C01A7B
:10165000524183098B4201D38B01C01A5241430985
:101660008B4201D34B01C01A524103098B4201D373
:101670000B01C01A5241C3088B4201D3CB00C01AE0
:10168000524183088B4201D38B00C01A5241430858
:101690008B4201D34B00C01A5241411A00D201467D
:1016A000524110467047FFE701B5002000F0F0F806
:1016B00002BDC0460029F7D076E7704703460B43CA
:1016C0007FD4002243088B4274D303098B425FD33B
:1016D000030A8B4244D3030B8B4228D3030C8B4267
:1016E0000DD3FF22090212BA030C8B4202D312124D
:1016F000090265D0030B8B4219D300E0090AC30B22
:101700008B4201D3CB03C01A5241830B8B4201D3CE
:101710008B03C01A5241430B8B4201D34B03C01AB7
:101720005241030B8B4201D30B03C01A5241C30A2F
:101730008B4201D3CB02C01A5241830A8B4201D3A0
:101740008B02C01A5241430A8B4201D34B02C01A8A
:101750005241030A8B4201D30B02C01A5241CDD22F
:10176000C3098B4201D3CB01C01A524183098B427A
:1017700001D38B01C01A524143098B4201D34B0163
:10178000C01A524103098B4201D30B01C01A5241C6
:10179000C3088B4201D3CB00C01A524183088B424D
:1017A00001D38B00C01A524143088B4201D34B0036
:1017B000C01A5241411A00D20146524110467047A8
:1017C0005DE0CA0F00D04942031000D340425340AD
:1017D00000229C4603098B422DD3030A8B4212D36D
:1017E000FC22890112BA030A8B420CD3890192119F
:1017F0008B4208D3890192118B4204D389013AD0DC
:10180000921100E08909C3098B4201D3CB01C01AB0
:10181000524183098B4201D38B01C01A52414309C3
:101820008B4201D34B01C01A524103098B4201D3B1
:101830000B01C01A5241C3088B4201D3CB00C01A1E
:10184000524183088B4201D38B00C01A5241D9D236
:1018500043088B4201D34B00C01A5241411A00D2B7
:101860000146634652415B10104601D34042002BB3
:1018700000D54942704763465B1000D3404201B532
:10188000002000F005F802BD0029F8D016E77047E7
:101890007047C0460C488546002103E00B4B5B585F
:1018A000435004310A480B4B42189A42F6D30A4A75
:1018B00002E0002313600432084B9A42F9D3FFF789
:1018C000ADFAFEF7AAFCFEE700100020041900089C
:1018D000000000209400002094000020D409002083
:1018E000FEE70000464F4F4241520A000000000050
:1018F00000000000010203040607080900000000C0
:0419000001020304D9
:1019040000127A000004004000200040002800403B
:10191400002C0040003000400054004000700040A3
:101924000000014000040140002401400827014058
:1019340008270140002C01400030014000380140DC
:1019440000440140004801400058014000000240AA
:10195400080002401C0002403000024044000240E3
:10196400580002400020024000F8FF1F001002400F
:10197400003002400000004800040048000800480D
:10198400000C00480014004800ED00E010E000E006
:0419940000E100E08E
:040000050800189542
:00000001FF
